:020000040000FA
:10000000E70A53087A08750862085208A2086B08C4
:1000100061080D080A0828086308290820084B0809
:1000200094086E0869086708200849086D08720876
:1000300065082C08200832083008300830082E08DF
:10004000170646055A03E2014604FE084604FE0868
:100050004604FE08460400084604FE084604FE085E
:100060004604FE084604000846048008460480084A
:100070004604FE0846047E084604FE08460480083E
:100080004604FE0846047E084604FE08460480082E
:100090004604FE0846047E084604FE08460480081E
:1000A00046048008460400084604BE08460480084A
:1000B0004604BC08460400084604B8084604800804
:1000C0004604B008460400084604A0084604800818
:1000D0004604800846040008460480084604800858
:1000E0004604800846040008E201000802080408EB
:1000F00008081008200840088108170646055A031A
:10010000E2014604C2084604C4084604C80846047E
:10011000D0084604E0084604C20802084605900AD2
:100120000000460466068E0A6607940A0008020C60
:1001300026003700F80C0600880C02008D093C00F0
:10014000290C3800060C3900280C30000A0C31004C
:10015000050C3200480C33000008FF0C340000008E
:10016000F402AF0A00000008AD09AD091C023B0013
:10017000430600084605AD09AD094604AD09AD09C1
:10018000FB02BA0AAD09AD09AD09AD090008FF0CC3
:10019000340066061D05000066061D05F402C90A46
:1001A000000866060008AD09AD097C00080C3B009C
:1001B0001D044605C709C7094604C709C709BC028B
:1001C0001D060008FB02D90A070C7C0100089709EC
:1001D000D109AD09AD09AD09AD09B4091C02740915
:1001E00035008E09000C7D09360046045002D80106
:1001F000170646053A0003040000460420091706C6
:10020000460555015601170446044307170517060E
:10021000460537044306370546041702260017062D
:1002200046053D04D000F80E460443063D0517067A
:1002300046058C0C3D068A0C460434000000170667
:100240004605F0023F0B00004604280C300017065C
:100250004605F102450B000046040A0C3100170662
:100260004605F2024B0B00004604050C320017064F
:100270004605F302510B020C260006020300460459
:10028000410B17064605440B00004604470B1706B2
:1002900046054A0B000046044D0B17064605500B59
:1002A000000046045202D901170646053A0003042D
:1002B000000046047D091706460536005F0B46041C
:1002C000610B17064605F4025F0B00004604680B3D
:1002D000170646050000F50AFF0FFF0FFF0FFF0F7F
:1002E000FF0FFF0FFF0FFF0FFF0FFF0FFF0FFF0F9E
:1002F000FF0FFF0FFF0FFF0FFF0FFF0FFF0FFF0F8E
:10030000FF0FFF0FFF0FFF0FFF0FFF0FFF0FFF0F7D
:10031000FF0FFF0FFF0FFF0FFF0FFF0FFF0FFF0F6D
:10032000FF0FFF0FFF0FFF0FFF0FFF0FFF0FFF0F5D
:10033000FF0FFF0FFF0FFF0FFF0FFF0FFF0FFF0F4D
:10034000FF0FFF0FFF0FFF0FFF0FFF0FFF0FFF0F3D
:10035000FF0FFF0FFF0FFF0FFF0FFF0FFF0FFF0F2D
:10036000FF0FFF0FFF0FFF0FFF0FFF0FFF0FFF0F1D
:10037000FF0FFF0FFF0FFF0FFF0FFF0FFF0FFF0F0D
:10038000FF0FFF0FFF0FFF0FFF0FFF0FFF0FFF0FFD
:10039000FF0FFF0FFF0FFF0FFF0FFF0FFF0FFF0FED
:1003A000FF0FFF0FFF0FFF0FFF0FFF0FFF0FFF0FDD
:1003B000FF0FFF0FFF0FFF0FFF0FFF0FFF0FFF0FCD
:1003C000FF0FFF0FFF0FFF0FFF0FFF0FFF0FFF0FBD
:1003D000FF0FFF0FFF0FFF0FFF0FFF0FFF0FFF0FAD
:1003E000FF0FFF0FFF0FFF0FFF0FFF0FFF0FFF0F9D
:0E03F000FF0FFF0FFF0FFF0FFF0FFF0FFF0F9D
:0203FE00FF0FEF
:08040000FF0FFF0FFF0FFF0FBC
:021FFE00E00FF2
:00000001FF
